:0200000059287D
:10000800A000030EA1000408A20083128B1C2D2857
:10001800A4011430240203181328A40A0D28A301EC
:100028000730230203182828A90CA9130519A917B2
:10003800A4010C30240203182328A40A1D28000058
:1000480000000000A30A1428A90CA9130519A91770
:100058008B1022088400210E8300A00E200E0900B8
:10006800A7008A0127081F39820720342034533417
:100078007034613472346B34463475346E342E34D3
:1000880063346F346D3400342034203420345334D6
:10009800653472344C344334443420347634313447
:1000A8002E34303400340034003483128320831219
:1000B800630000002908FE3A031D6D286300000054
:1000C800290E0F39033A03195C28290812218312D3
:1000D8005C282908E420AA0A2A08103A031D7A286D
:1000E800C03012214030AA0083125C282A08503AF6
:1000F800031D5C2880301221AA0183125C28073076
:1001080099008501043083168500831287018316C0
:100118008701831285100710DC30A5000530A60082
:100128004F21071187110716871687148710643027
:10013800A500A6014F2107118711071687168714F6
:1001480087106430A500A6014F21071187110716F3
:100158008716871487100A30A500A6014F210711BA
:10016800871107168712871487100C301221013067
:1001780083121221A50183124121C03012210F30B0
:10018800A50083124121C430A5000930A6004F21E3
:1001980001301221AA0101130B168B1708003C30FD
:1001A80083168700831285100714871428100719EF
:1001B80028148710871487100310281803140800C0
:1001C800A700D3200318E528071085148316870194
:1001D8008312A71F0711A71B0715271F8711271BA6
:1001E8008715A71E0712A71A0716271E8712271A90
:1001F800871687148710A71D0711A7190715271D2C
:10020800871127198715A71C0712A7180716271C77
:10021800871227188716871487100800A500D3208F
:100228000318132907108510831687018312A51F49
:100238000711A51B0715251F8711251B8715A51E47
:100248000712A51A0716251E8712251A871687145E
:100258008710A51D0711A5190715251D8711251933
:100268008715A51C0712A5180716251C871225181F
:1002780087168714871083160800A6012608250705
:100288003420003A03194E29260825073420E42093
:10029800A60A422908002508260403196129A7018E
:1002A800A71B5A296C30270203185C29A70A54296E
:0C02B800A503250A0319A6034F2908001E
:02400E009431EB
:00000001FF
